:0A0CF60000010202030304040505D7
:10060B00E4F513F512F511F510C203C200C202C2D4
:10061B000112174E1207B87E107F008E4A8F4B7552
:10062B00521075531275481075491C755010755141
:10063B004A755410755578EE54E0700302075275E5
:10064B0014007515808E168F17C374A29FFF74103C
:10065B009ECF2402CF3400FEE48F0F8E0EF50DF5E6
:10066B000CF50BF50AF509F508AF0FAE0EAD0DAC99
:10067B000CAB0BAA0AA909A808C31212915026E5C4
:10068B0015250BF582E514350AF58374CDF0E50BD2
:10069B002401F50BE4350AF50AE43509F509E435CF
:1006AB0008F50880C4E4F50BF50AF509F508AF0F5A
:1006BB00AE0EAD0DAC0CAB0BAA0AA909A808C31260
:1006CB0012915031AE0AAF0BE5172FF582E5163EAE
:1006DB00F583E0FDE5152FF582E5143EF583EDF08E
:1006EB00EF2401F50BE43EF50AE43509F509E43591
:1006FB0008F50880B985144A85154B74002480FFD2
:10070B00741034FFFEC3E5539FF553E5529EF5522B
:10071B00C3E54D9FF54DE54C9EF54CC3E54F9FF55D
:10072B004FE54E9EF54EC3E5499FF549E5489EF5CD
:10073B0048C3E5519FF551E5509EF550C3E5559FD4
:10074B00F555E5549EF554D2E843D82090E668E081
:10075B004409F090E65CE0443DF0D2AF90E680E0D7
:10076B0020E105D20812153090E680E054F7F053E3
:10077B008EF8C2033001051203E7C20130032912C0
:10078B0019045024C2031216E220001690E682E0F0
:10079B0030E704E020E1EF90E682E030E604E02071
:0D07AB00E0E41215B91219061211B980C749
:1003E70090E6B9E07003020498147003020515241F
:1003F700FE700302059824FB700302049214700335
:1004070002048C146073146076240560030205F7F8
:10041700121908400302060390E6BBE024FE60229F
:1004270014603324FD601114602224067048E54AE5
:1004370090E6B3F0E54B8037E55290E6B3F0E5532D
:10044700802DE54C90E6B3F0E54D8023E54E90E630
:10045700B3F0E54F801990E6BAE0FF1215E5AA065A
:10046700A9077B01EA494B600DEE90E6B3F0EF90E8
:10047700E6B4F00206030205FC1217E802060312AF
:10048700187F0206031213800206031217D602060C
:100497000312190A400302060390E6B8E0247F60BE
:1004A7001514601924027063A200E43325E0FFA24B
:1004B70002E4334F8041E490E740F0803F90E6BC90
:1004C700E0547EFF7E00E0D394807C0040047D01F1
:1004D70080027D00EC4EFEED4F24F6F582740C3E53
:1004E700F583E493FF3395E0FEEF24A1FFEE34E6B6
:1004F7008F82F583E0540190E740F0E4A3F090E6A3
:100507008AF090E68B7402F00206030205FC1219CA
:100517000C400302060390E6B8E024FE60162402AE
:10052700600302060390E6BAE0B40105C2000206C2
:10053700030205FC90E6BAE0705590E6BCE0547EF5
:10054700FF7E00E0D394807C0040047D0180027D23
:1005570000EC4EFEED4F24F6F582740C3EF583E475
:1005670093FF3395E0FEEF24A1FFEE34E68F82F58B
:1005770083E054FEF090E6BCE05480131313541F3D
:10058700FFE0540F2F90E683F0E04420F0806D8069
:100597006412190E506690E6B8E024FE6019240232
:1005A700705A90E6BAE0B40104D200804F90E6BAE0
:1005B700E064026047803E90E6BCE0547EFF7E0028
:1005C700E0D394807C0040047D0180027D00EC4EE6
:1005D700FEED4F24F6F582740C3EF583E493FF336A
:1005E70095E0FEEF24A1FFEE34E68F82F5838008C5
:1005F700120080500790E6A0E04401F090E6A0E0EA
:030607004480F03C
:01060A0022CD
:030033000218F0C0
:0418F00053D8EF32A8
:10174E00758CE0758AC0E58954F04401F589758E73
:08175E0003D28CD2A9D2AF2204
:03000B00020DB82B
:100DB800C0E0C0F0C083C082C0D075D000C000C001
:100DC80001C002C003C004C005C006C007758CE09E
:100DD800758AC0D28CE47F607EEAFDFCAB47AA46E8
:100DE800A945A844C31212915019AF47AE46AD4564
:100DF800AC44EF2401F547E43EF546E43DF545E40F
:100E08003CF544E47F01FEFDFCAB47AA46A945A892
:100E180044C31212917008E5A054F02531F5A0E5FD
:100E28002B2401FFE4352AFEE4FCFDAB47AA46A9C2
:100E380045A844C3121291700553A0F0C28CD00784
:100E4800D006D005D004D003D002D001D000D0D035
:090E5800D082D083D0F0D0E0324A
:1010000012010002000000401816036000000102F7
:1010100000010A06000200000040010009022E0043
:1010200001010080FA0904000004FF000000070528
:1010300001024000000705820200020007050202CB
:101040000002000705810240000009022E00010194
:101050000080FA0904000004FF00000007050102F7
:10106000400000070582024000000705020200025E
:101070000007058102400000040309041003510029
:10108000480059002D00430043004400160351005E
:10109000480059002D003800500052004F00200039
:0410A000200000002C
:100AB3006080280001040202020202070000000213
:100AC300000002001332120A080C080000000000A4
:100AD3000000003F010402020202020700000002BC
:100AE3000000020013320A12100C0800000000007C
:100AF3000000003F033A030303030307000000025F
:100B0300000002001332120A080C08000000000063
:100B13000000003F035A030303030307000000021E
:100B23000000020013320A12100C0800000000003B
:100B33000000003F60242887000000000000000040
:100B430000000000000000000000000000000000A2
:100B53000000000000000000000000004728808023
:060B6300000000CA4E0074
:100C3A0090E60174CAF090E6F574FFF0902880E01F
:100C4A0090E6F3F0902881E090E6C3F0902882E0E5
:100C5A0090E6C1F0902883E090E6C2F0902885E003
:100C6A0090E6C0F0902886E090E6F4F075AF07743D
:100C7A0028F59A7400F59B759DE4E4F59EFF90E6CD
:100C8A007BE090E67CF00FBF80F490E67174FFF091
:100C9A00F5B490E672E04480F043B680000000E4C8
:100CAA0090E6C4F000000090E6C5F0902887E09036
:100CBA00E6C6F0902888E090E6C7F0902889E09090
:100CCA00E6C8F090288AE090E6C9F090288BE09078
:100CDA00E6CAF090288CE090E6CBF090288DE09060
:0B0CEA00E6CCF090288EE090E6CDF004
:010CF50022DC
:03004300020D00AB
:03005300020D009B
:100D0000021766000217AC000217960002177E0059
:100D10000213FA000213BD00020FFF0002191000B7
:100D20000219110002191200020FA200020F07009F
:100D300002191300021914000219150002191600F5
:100D400002191700021910000219180002191900DF
:100D500002191A0002191B0002191C0002191D00B9
:100D600002191E00021910000219100002191000C9
:100D700002191F0002192000021921000219220085
:100D80000219230002192400021925000219260065
:100D900002192700021928000219290002192A0045
:100DA00002192B0002192C0002192D0002192E0025
:080DB00002192F0002193000A6
:1015B90090E682E030E004E020E60B90E682E0303D
:1015C900E119E030E71590E680E04401F07F147EF0
:0C15D9000012133A90E680E054FEF0226D
:1016E20090E682E044C0F090E681F043870100007A
:0416F20000000022D2
:1015300030080990E680E0440AF0800790E680E0F9
:101540004408F07FDC7E0512133A90E65D74FFF0EC
:0F15500090E65FF05391EF90E680E054F7F022C1
:0215E500A90754
:1015E700AE54AF558F828E83A3E064037017AD01AD
:1015F70019ED7001228F828E83E07C002FFDEC3E77
:09160700FEAF0580DF7E007F00CC
:0116100022B7
:10133A008E1E8F1F90E600E054187012E51F2401DC
:10134A00FFE4351EC313F51EEF13F51F801590E653
:10135A0000E05418FFBF100BE51F25E0F51FE51E3E
:10136A0033F51EE51F151FAE1E7002151E4E6005D1
:06137A001216F680EE22BF
:1016F6007400F58690FDA57C05A3E582458370F907
:0117060022C0
:100B6900C18502230000022E1040C1070440000085
:020B790000007A
:08163D0090E679F07F057E00C4
:101645008E1E8F1FE51F451E60177F957E001213A6
:1016550023000000000000E51F151F70E7151E8020
:02166500E3227E
:1007B80090E600E054E74410F000000000000090CC
:1007C800E61074A0F000000090E60B7401F090E6CB
:1007D8001274E0F0000000E490E613F000000090CE
:1007E800E614F000000090E615F000000090E6180E
:1007F800740CF000000090E6D27402F090E60474E5
:1008080080F00000007402F0000000E4F000000036
:10081800120C3AE490E671F075B4FF90E672F07548
:10082800B6FF75B1FF90E670F075B2FFC28CD28743
:10083800D28512180C75230275240000000090E67A
:100848001074A0F000000000000090E611F0000015
:100858000090E65EE04408F0000000E490E68DF0C9
:1008680090E65EE04404F0000000E490E68FF012A9
:10087800158C5380FE7F9A7E0012184075280075EB
:1008880029B4753B01753C90752E10752FB8753ECF
:1008980006753F2C12188F90E67AE054FEF0E4FDBE
:1008A8007F9012149A7F647E0012133A7DFF7F4274
:1008B80012149A7F647E0012133A7D827F4E1214BE
:1008C8009A7532FF75358290E782E532F090E781BC
:0908D800E535F01218EB02180CD2
:10113000E535D3940040037532FF90E678E04480B3
:10114000F0749112163D90E679E090E7C0121640D7
:1011500090E679E090E7C112164090E679E090E7DA
:10116000C212164090E679E090E7C312164090E66E
:1011700078E0444012164090E678E04480F07442F3
:1011800012163D90E679E53212164090E678E0447A
:101190004012164090E678E04480F090E679744E74
:1011A00012164090E679E53512164090E678E04454
:0911B00040F07F057E00021645A7
:1011B900E5432401F543E43542F542E43541F5417F
:1011C900E43540F540E47FE87E03FDFCAB43AA42E9
:1011D900A941A840C31212917006FD7F9012149A7A
:1011E9007FA07E867D017C00AB43AA42A941A8402D
:1011F900C31212917009120FFA1211301218EB7FF3
:10120900407E0D7D037C00AB43AA42A941A840D38F
:101219001212914009E4F543F542F541F5403004D5
:0712290003120B7CC204223A
:02190400D322EC
:02190600D322EA
:02190800D322E8
:1013800090E680E030E71800000090E6207402F05C
:10139000000000E490E621F0000000D20580160075
:1013A0000000E490E620F000000090E6217440F098
:0D13B000000000C20590E6BAE0F539D32236
:1017D60090E740E539F0E490E68AF090E68B04F075
:0217E600D3220C
:08187F0090E6BAE0F527D32240
:1017E80090E740E527F0E490E68AF090E68B04F075
:0217F800D322FA
:02190A00D322E6
:02190C00D322E4
:02190E00D322E2
:10008000E4F518F51990E6B9E0244B606B147003A1
:1000900002024624F4700302027E24FD7003020271
:1000A000C914700302032D24FD7003020362241699
:1000B00060030203E3E490E68AF090E68BF090E6BA
:1000C000A0E020E1F990E68BE0F518E4F5B5F5B392
:1000D00090E60174CAF0E490E6C3F090E6C2F0D274
:1000E0000400000090E6047480F00000007402F048
:1000F000000000E4F00203E5E490E68AF090E68B6D
:10010000F090E6A0E020E1F990E68BE0F518D394BA
:100110003F4024E4F51974402519F582E434E7F5ED
:1001200083E0FF74AB2519F582E43428F583EFF002
:100130000519E519B440DF7F9A7E00121840902817
:10014000ABE0FF7E001218499028ABE0FF7E001262
:1001500018529028ABE0FF7E0012185B9028ACE0AC
:1001600075F004A4FFAEF01218649028ACE075F0AE
:1001700004A4FFAEF012186D9028ACE075F004A452
:10018000FFAEF01218769028B0E0C394025013909E
:1001900028CCE090E6C07005744EF08016749CF098
:1001A00080119028CCE090E6C07005749FF0800329
:1001B000749DF09028CEE0F5369028CBE0F5349091
:1001C00028CFE0F53A9028D9E0F533A3E0FEA3E08C
:1001D0007C002400F526EC3EF5259028B1E0F530B2
:1001E000E53070037530019028B6E0FEA3E07C0096
:1001F0002400F529EC3EF528A3E0FEA3E02400F559
:100200003CEC3EF53B9028B2E0FEA3E02400F52F45
:10021000EC3EF52EA3E0FEA3E02400F53FEC3EF516
:100220003E9028BCE0FEA3E02400F538EC3EF53714
:100230009028BAE0FEA3E02400F52DEC3EF52CE476
:10024000FD7F9002035CE4F51974AB2519F582E497
:100250003428F583E0FF74402519F582E434E7F58E
:1002600083EFF00519E519B40ADF000000E490E619
:100270008AF000000090E68B740AF00203E590E734
:100280004074ABF0A37408F0A3740CF0A37426F0D0
:10029000A37407F0A374EEF0A37401F0A37403F049
:1002A000A37453F0300505E4A3F0800690E7497489
:1002B000FFF0000000E490E68AF000000090E68B7A
:1002C000740AF012158C0203E590E678E04480F0A1
:1002D00090E6797491F07F647E0012132390E679A2
:1002E000E090E740F07F647E0012132390E679E00F
:1002F00090E741F07F647E0012132390E679E0904E
:10030000E742F07F647E0012132390E679E090E7E5
:1003100043F090E678E04440F0000000E490E68A84
:10032000F000000090E68B7404F00203E5E490E630
:100330008AF090E68BF090E6A0E020E1F990E68B61
:10034000E0F518D3940150030203E590E741E0FD86
:100350007F4212149A90E740E0FD7F4E12149A02F9
:1003600003E5E490E68AF090E68BF090E6A0E020CA
:10037000E1F990E68BE0F518D39401406890E740EE
:10038000E05480C4131313540124FF92A3E054409B
:10039000C41313540324FF92A2E05420C41354073F
:1003A00024FF92A1E05410C4540F24FF92A0A3E0B4
:1003B00075F00AA4FFAEF012133A90E740E054083B
:1003C000131313541F24FF92A3E054041313543F38
:1003D00024FF92A2E05402C31324FF92A1E01392DF
:0603E000A08002D322C33D
:0103E60022F4
:10176600C0E0C083C082D2015391EF90E65D740160
:08177600F0D082D083D0E032F4
:10179600C0E0C083C0825391EF90E65D7404F0D040
:0617A60082D083D0E03286
:1017AC00C0E0C083C0825391EF90E65D7402F0D02C
:0617BC0082D083D0E03270
:1013FA00C0E0C083C08285504C85514D854D8285A1
:10140A004C83A37402F085484E85494F854F8285E7
:10141A004E83A37407F05391EF90E65D7410F0D0F9
:06142A0082D083D0E03205
:10177E00C0E0C083C082D2035391EF90E65D74083F
:08178E00F0D082D083D0E032DC
:1013BD00C0E0C083C08290E680E030E72085484CD5
:1013CD0085494D854D82854C83A37402F085504E21
:1013DD0085514F854F82854E83A37407F05391EF4E
:0D13ED0090E65D7420F0D082D083D0E03215
:010FFF0032BF
:0119100032A4
:0119110032A3
:0119120032A2
:100FA200C0E0C0F0C083C082C0D075D000C000C015
:100FB20001C002C003C004C005C006C007C2AF1210
:100FC2000FFA00000090E68F7404F00000005391C5
:100FD200EF90E65FE04404F01218EBD2AFD007D0F6
:100FE20006D005D004D003D002D001D000D0D0D09A
:080FF20082D083D0F0D0E03280
:100F0700C0E0C083C082C0D075D000C004C006C096
:010F170007D2
:100F1800C2AF90E6A1E020E1F990E780E014601408
:100F280024F8601E240C604624FE60461470487540
:100F38002200804390E782E0F53290E781E0F535C2
:100F48008035D28C90E781E0540FF531A3E0FEA301
:100F5800E07C002400FFEC3EC313F52AEF13F52BC9
:100F68007547007546007545007544008009C28CB8
:100F78008005752200D20600000090E68DE4F0534B
:0B0F880091EF90E65FE04408F0D2AF6C
:0F0F9300D007D006D004D0D0D082D083D0E032A7
:0119130032A1
:0119140032A0
:01191500329F
:01191600329E
:01191700329D
:01191800329C
:01191900329B
:01191A00329A
:01191B003299
:01191C003298
:01191D003297
:01191E003296
:01191F003295
:011920003294
:011921003293
:011922003292
:011923003291
:011924003290
:01192500328F
:01192600328E
:01192700328D
:01192800328C
:01192900328B
:01192A00328A
:01192B003289
:01192C003288
:01192D003287
:01192E003286
:01192F003285
:011930003284
:0609E9008F1A8C1B8D1C0F
:1009EF00531A0753A0BF7F0A7E00121323E4F51D8D
:1009FF00F51EC37402951EFFE51AA807088002C3EF
:100A0F0013D8FC30E00543A020800353A0DF7F0AFA
:100A1F007E0012132343A0107F0A7E00121323536C
:100A2F00A0EF7F0A7E00121323051EE51E7002053C
:100A3F001DC39403E51D6480948040B6E4F51DF555
:100A4F001EC37409951EFFE51CAE1BA80708800581
:100A5F00CEC313CE13D8F930E00543A02080035343
:100A6F00A0DF7F0A7E0012132343A0107F0A7E00AF
:100A7F0012132353A0EF7F0A7E00121323051EE5E6
:100A8F001E7002051DC3940AE51D6480948040B159
:100A9F0043A0407F0A7E0012132353A0BF7F0A7E1C
:040AAF00000213230B
:09184000AD07AC06E4FF0209E962
:09184900AD07AC067F040209E9B9
:09185200AD07AC067F050209E9AF
:09185B00AD07AC067F060209E9A5
:09186400AD07AC067F010209E9A1
:09186D00AD07AC067F020209E997
:09187600AD07AC067F030209E98D
:10149A008D1AAD0790E678E04480F090E679EDF099
:1014AA007F647E0012132390E679E51AF07F647E4A
:1014BA000012132390E678E04440F07F647E000235
:0214CA001323EA
:1012EF007E001213231218027F147E001213231292
:1012FF0018F47F037E001213231219007F027E0061
:10130F001213231218227F027E0012132312183693
:04131F007F027E00CB
:10132300EF7803C333CE33CED8F9FFEF4E6007EF28
:071333001F70F81E80F52277
:0718970053B1EF53B1BF2272
:07189E0053B1EF43B14022FA
:0718A50043B11043B14022E2
:0718AC0053B1FE53B1FB2212
:0718B30053B1FE43B1042212
:0718BA0043B10143B1042218
:0418F40053B1F722D3
:0418F80043B10822CE
:0418FC0053B17F2243
:0419000043B180224D
:0718C10053B1EF53B1DF2228
:0718C80053B1EF43B12022F0
:0718CF0043B11043B12022D8
:0718D60053B1FE53B1FD22E6
:0718DD0053B1FE43B10222EA
:0718E40043B10143B10222F0
:0A17C20012180C7F0A7E0012132398
:0A17CC0053B1EF53B1BF53B1DF2258
:0A18180053B1FE53B1FB53B1FD22A2
:0A18220053B1EF43B14043B120225F
:0817FA007E00121323121822D5
:0A18020053B1FE43B10443B10222CA
:0A182C0043B11043B14043B1202244
:0A18360043B10143B10443B10222A3
:0C180C001218221218F81218360218FCEC
:10172B001217C27F031217FA12182C1218187F0304
:10173B001212EF1218FC12131F1218F87F147E00EE
:03174B0002132363
:101667001217C27F081217FA7F017E001213231286
:10167700182C1218187F021212EF1218FC12131FDF
:0A1687001218F87F147E00021323EE
:1014CC0012180C5380FE7F017E0012132312180297
:1014DC0012131F12182C12131F1218F47F0212135E
:1014EC00031218FC7F147E001213231218F8438089
:0214FC000122CB
:10155F0012180C12131FE4FFFE12180212182C128D
:10156F0018F41219001218221218361218FC121839
:0C157F00F80FBF00010EBE03E0BFF7DD57
:01158B00223D
:08188700C28512131FD2852255
:10158C00C283E4F51AF51BD2827F1E7E0012133A39
:10159C00C2827F1E7E0012133A051BE51B700205EA
:0C15AC001AC39405E51A6480948040DBAB
:0115B8002210
:050FFA00C283C2822247
:0518EB00D283D282222D
:011931002293
:011932002292
:100E61001218F812182CE52D452C7003121887E57D
:100E710034B40102C287121931E536707575220149
:100E81009028ADE075F040A485F01CF51DAF227EE1
:100E910000AC1CAD1D12127FD3EF9400EE94004004
:100EA100147FC47E03121645121130E51D151D7005
:100EB100DC151C80D89028AEE0751C00F51DAF2212
:100EC1007E00AC1CAD1D12127FD3EF9400EE940096
:100ED10040147FC47E00121645121130E51D151D08
:100EE10070DC151C80D89028AFE0FF7E0012133A09
:100EF1008009752201E522640160FA121932E53494
:050F0100B40102D287DB
:010F060022C8
:10161100AD07AC06D3ED9400EC9400401E00000031
:10162100EE90E6D0F0000000ED90E6D1F000000071
:0C16310075BB04000000E5BB30E7FB22A5
:0212A200AC0698
:1012A40090E6C0E0FBE490E618F090E6C0744EF0DF
:1012B400EC90E6D0F0000000EF90E6D1F0000000E2
:1012C40075BB04000000E5BB30E7FB90E6047480C6
:1012D400F00000007402F0000000E4F00000009050
:0A12E400E618740CF090E6C0EBF081
:0112EE0022DD
:10169100AD07AC06000000ED25E0EC3390E6D0F09C
:1016A100000000ED25E090E6D1F000000075BB04DC
:0916B100000000E5BB30E7FB225C
:10170700E53A700E120E61E52D452C701112155F2A
:10171700800CE52D452C700312155F120E61121710
:041727002BD2862219
:100B7C001218EBC206121707120FFA300603020CFA
:100B8C0039E4F51AF51BC3E51B9529E51A95285090
:100B9C000D1214CC051BE51B70EC051A80E8E5332F
:100BAC00D39400400EAF337E00AC2EAD2F12127FCB
:100BBC001212A2D3E5269400E52594004007AF2637
:100BCC00AE25121691E4F518F519C3E519953FE514
:100BDC0018953E502C1216BAE4F51AF51BC3E51BFA
:100BEC0095307480F8651A98500D1214CC051BE5DD
:100BFC001B70EA051A80E60519E51970CD051880F9
:100C0C00C9E4F51AF51BC3E51B953CE51A953B5059
:100C1C000D1214CC051BE51B70EC051A80E812189C
:0D0C2C00F812182CC286AF38AE3712161120
:010C39002298
:1016BA00000000E52F25E0E52E3390E6D0F000008B
:1016CA0000E52F25E090E6D1F000000075BB04008C
:0816DA000000E5BB30E7FB2234
:08188F00E4F55BD2E9D2AF22BF
:1014300090E678E020E6F9C2E990E678E04480F0B2
:10144000EF25E090E679F090E678E030E0F990E67C
:1014500078E04440F090E678E020E6F990E678E025
:0614600030E1D6D2E922C2
:1014FE00A90790E678E020E6F9E55B702390E678A0
:10150E00E04480F0E925E090E679F08D56AF03A92E
:10151E00077557018A588959E4F55A755B01D3222C
:02152E00C322D6
:10146600A90790E678E020E6F9E55B702590E67836
:10147600E04480F0E925E0440190E679F08D56AF2E
:1014860003A9077557018A588959E4F55A755B030C
:04149600D322C32278
:03004B000208E1C7
:1008E100C0E0C083C082C085C084C086758600C058
:1008F100D075D000C000C001C002C003C006C0074F
:1009010090E678E030E206755B060209CB90E67866
:10091100E020E10CE55B64026006755B070209CB30
:10092100E55B24FE605F14603624FE70030209BC9F
:1009310024FC70030209C8240860030209CBAB57E9
:10094100AA58A959AF5A055A8F82758300121230DD
:1009510090E679F0E55A65567070755B05806B908D
:10096100E679E0AB57AA58A959AE5A8E8275830031
:1009710012125D755B02E5566401704E90E678E0F7
:100981004420F08045E55624FEB55A0790E678E00C
:100991004420F0E55614B55A0A90E678E04440F058
:1009A100755B0090E679E0AB57AA58A959AE5A8E0B
:1009B1008275830012125D055A800F90E678E0443B
:1009C10040F0755B008003755B005391DFD007D069
:1009D10006D003D002D001D000D0D0D086D084D0B0
:0809E10085D082D083D0E03202
:030000000210A447
:0C10A400787FE4F6D8FD75815B0210EB4C
:10123000BB010CE58229F582E5833AF583E0225073
:1012400006E92582F8E622BBFE06E92582F8E222BD
:0D125000E58229F582E5833AF583E49322D7
:10125D00F8BB010DE58229F582E5833AF583E8F0C7
:10126D00225006E92582C8F622BBFE05E92582C873
:02127D00F2225B
:10127F00EF8DF0A4A8F0CF8CF0A428CE8DF0A42E83
:02128F00FE223D
:10129100EB9FF5F0EA9E42F0E99D42F0E89C45F0B3
:0112A100222A
:1010B00002060BE493A3F8E493A34003F68001F245
:1010C00008DFF48029E493A3F85407240CC8C33341
:1010D000C4540F4420C8834004F456800146F6DF10
:1010E000E4800B0102040810204080900AB3E47EE3
:1010F000019360BCA3FF543F30E509541FFEE49305
:10110000A360010ECF54C025E060A840B8E493A3CB
:10111000FAE493A3F8E493A3C8C582C8CAC583CAF6
:10112000F0A3C8C582C8CAC583CADFE9DEE780BEAE
:010B7B000079
:00000001FF
